:100000000C942E000C9449000C9449000C94490067
:100010000C9449000C9449000C9449000C9449003C
:100020000C9449000C9449000C9449000C9449002C
:100030000C9449000C9449000C9449000C9449001C
:100040000C9449000C9449000C9449000C9449000C
:100050000C9449000C9449000C94490011241FBED3
:10006000CFEFD0E1DEBFCDBF11E0A0E0B1E0EEEC1C
:10007000F0E002C005900D92A030B107D9F711E071
:10008000A0E0B1E001C01D92A030B107E1F70C94EF
:1000900057000C9400009C0106C080EF90E001978F
:1000A000F1F72150304021153105B9F70895CFEF10
:1000B000D0E1DEBFCDBF3D9A459882E390E00E943B
:0E00C0004B00459A82E390E00E944B00F5CF82
:00000001FF
